:1000000019C020C01FC01EC01DC01CC01BC01AC00C
:1000100019C018C01DC017C019C014C013C012C029
:1000200011C010C00FC00EC00DC00CC00BC00AC064
:1000300009C008C011241FBECFEFD2E0DEBFCDBF84
:10004000DCD0EAC2DDCF3BB828B8189525B81895A2
:10005000F09A3BB828B825B846BA18958895F09B11
:10006000FDCFF09808951F93CF93DF93EC019B0190
:1000700019854F81E12FF0E0EE9FC001EF9F900DB9
:10008000FE9F900D11248E0F9F1F642F70E099D258
:10009000769567952617370728F4411798F4141BAF
:1000A000198710C05E81151768F4852F90E08E1BAC
:1000B0009F0B242F30E08217930714F4598702C056
:1000C000410F4987DF91CF911F9108950F931F939F
:1000D000CF93DF93EC01888581FF2DC00C811D81BA
:1000E00080FF12C088819981B801681B790BCE010D
:1000F000BADF8985B801681B710928813981261703
:10010000370788F0188613C06A817B81601B710BEA
:10011000CE01A9DF8985B801680F711D2A813B8155
:100120006217730710F49B0104C081E08887198669
:10013000F1983D832C83DF91CF911F910F9108950A
:10014000FC019085892F91FF05C0118680958170F3
:10015000808702C092609087F1980895FC018085A5
:1001600081FF12C0759567958681680F711D6F3F7D
:10017000710519F014F06FEF70E06830710514F438
:1001800068E070E06683089594E0660F771F9A95A3
:10019000E1F72081318180FF14C082819381860F35
:1001A000971F2817390710F0C90101962CE98F33E2
:1001B000920710F08EE39CE9938382839583848376
:1001C0000895620F731F8FE16034780710F460E4C4
:1001D0007FE1828193816817790718F0BC01615033
:1001E000704071836083758364830895FC0124816A
:1001F000358136952795C90108955F928F929F9218
:10020000AF92BF92CF92DF92EF92FF920F931F9324
:10021000CF93DF9380E885BF8FEF84B98EE387B9F2
:1002200080EC8AB99FE3392E8FE38BB986E0482EA4
:10023000222489E1809381008FE19EE490938700DE
:100240008093860086E280936F0081E080937E0039
:1002500080B7806880BF80E480937C0080E091E07C
:1002600060E070E048E950E0C0D1809197018F3F95
:1002700019F08093660004C0809166008093970116
:10028000CC244FE143950AB01BB0900104261426FC
:100290001BB80AB8D49ED12CC49E1D0C60014A958F
:1002A00009B03BB92AB900940422C028469551F7F9
:1002B0001124789401EC502E88248A94982C11E013
:1002C000A12EB12C01C06701C9DE289A459A809100
:1002D0005E0190915F019695879590938B00809336
:1002E0008A008091040190910501969587959093DD
:1002F00089008093880080E091E0E8DE80E591E06D
:10030000E5DEACDE299A449A8091720190917301E6
:100310009695879590938B0080938A0080910E012B
:1003200090910F019695879590938900809388000E
:100330008AE091E0CBDE8AE591E0C8DE8FDE2A9A82
:10034000439A809168019091690196958795909361
:100350008B0080938A0080911801909119019695E5
:100360008795909389008093880084E191E0AEDEC8
:1003700084E691E0ABDE72DE2B9A429A8091900186
:10038000909191019695879590938B0080938A0028
:1003900080912201909123019695879590938900F1
:1003A000809388008EE191E091DE8EE691E08EDE12
:1003B00055DE2C9A419A80919001909191019695E9
:1003C000879590938B0080938A0080912C01909167
:1003D0002D0196958795909389008093880088E2F7
:1003E00091E074DE88E791E071DE38DE2D9A5E9A46
:1003F00080918601909187019695879590938B00C7
:1004000080938A0080914A0190914B01969587953F
:10041000909389008093880082E391E057DE82E820
:1004200091E054DE1BDE2E9A5F9A80917C019091C0
:100430007D019695879590938B0080938A0080919B
:1004400054019091550196958795909389008093DA
:1004500088008CE391E03ADE8CE891E037DE509240
:100460007A00FCDD2F9A8091680190916901969540
:10047000879590938B0080938A0090928900809258
:10048000880086E491E022DEE0E0F1E0808581FDF5
:100490001EC03A9621E0E639F207C0F3F99917C079
:1004A000C0E0D1E000E010E0C801AED0988189172B
:1004B00031F090BDF894FA9A7894F99A08C081E0E6
:1004C000C739D80721F021960F5F1F4FEDCF20913C
:1004D00078003091790010927A00F19B27C0B90121
:1004E000661977093901809196018F3040F42AE02E
:1004F000829FC001112480509F4F30DE1EC0759531
:1005000067957595679580919701680F711D6F3F8D
:10051000710519F014F06FEF70E077FF02C060E032
:1005200070E0609397016093660007C0C901805F27
:100530009140809710F4F19A3901EE244FE14395F0
:100540000AB01BB09001042614261BB80AB8F49E0A
:10055000F12CE49E1F0C70014A9509B03BB92AB9F1
:1005600000940422E028469551F711248601009555
:1005700010950E211F210115110509F4A4CEC0E02C
:10058000D0E0C5010C2E02C0880F991F0A94E2F733
:1005900080239123892B81F0C09396019E01CE0187
:1005A00063E0880F991F6A95E1F7220F331F820FCE
:1005B000931F80509F4FC4DD2196CF30D10509F79E
:1005C00082CEAA1BBB1B51E107C0AA1FBB1FA617E7
:1005D000B70710F0A61BB70B881F991F5A95A9F7EC
:1005E00080959095BC01CD010895DC01862FE82F00
:1005F000F999FECF12BC05C0E1BDF89AE39500B4AD
:100600000D924150C8F70895F999FECF12BC81BDF3
:0C061000F89A992780B50895F894FFCF60
:00000001FF
